:100000000C9496010C94BE010C94BE010C94BE019C
:100010000C94BE010C94BE010C94BE010C94BE0164
:100020000C94BE010C9437030C9419230C94CB212F
:100030000C94BE010C94BE010C94BE010C94BE0144
:100040000C94540A0C94BE010C94BE010C94BE0195
:100050000C94BE010C94BE010C94BE010C94E719E3
:100060000C94BE010C94C01E0C94031F0C94BE0192
:100070000C94BE010C94BE010C94BE010C94BE0104
:100080000C94BE010C94BE010C94BE010C94BE01F4
:100090000C94BE010C94BE010C94BE010C94BE01E4
:1000A0000C94BE010C94BE010C94BE018A129012F5
:1000B00096129D12AB12CD12EB12F01AF31AE61A39
:1000C000EA1A141B141B141BF71AFB1AFF1A051B40
:1000D000091B141B0F1B434C49206E6F7420617663
:1000E00061696C61626C652C2075736520636F6E4D
:1000F000666967757261746F72210000000002000A
:10010000080E0000030401000B00000000000000C6
:100110000000000000000000000408020110408000
:1001200040102040804080080204018040201002DE
:10013000011080102040400404040404030405025C
:100140000202020403020202020606060606060472
:100150000402020204000000002300260029002CF3
:10016000002F0000000000250028002B002E003189
:100170000000000000240027002A002D00300008A5
:100180000B0002020201000904000001020200004B
:1001900005240010010524010101042402060524A0
:1001A0000600010705810310004009040100020A4E
:1001B000000000070502024000000705830240001E
:1001C0000000C18081C112010002020000404123F1
:1001D000368000010102000112010002000000400F
:1001E0004123368000010102000118034100720022
:1001F0006400750069006E006F0020004C004C0028
:1002000043002203410072006400750069006E0023
:100210006F0020004C0065006F006E0061007200EE
:1002200064006F00040309040000000000000000E7
:100230002A2B280000000000000000000000000041
:1002400000000000000000002C9EB4A0A1A2A43475
:10025000A6A7A5AE362D3738271E1F20212223241E
:100260002526B333B62EB7B89F8485868788898ABA
:100270008B8C8D8E8F909192939495969798999A56
:100280009B9C9D2F3130A3AD350405060708090A54
:100290000B0C0D0E0F101112131415161718191A36
:1002A0001B1C1DAFB1B0B500090402000103000022
:1002B00000092101010001226500070584034000B7
:1002C0000105010902A1010901A100850105091922
:1002D000012903150025019503750181029501751A
:1002E00005810305010930093109381581257F751C
:1002F0000895038106C0C005010906A10185020514
:100300000719E029E7150025017501950881029577
:1003100001750881039506750815002565050719FF
:100320000029658100C0A11CF11FB52411241FBE46
:10033000CFEFDAE0DEBFCDBF12E0A0E0B1E0E6E152
:10034000FCE402C005900D92AA35B107D9F715E07B
:10035000AAE5B2E001C01D92A831B107E1F713E0B0
:10036000CCE2D3E004C02297FE010E947E25C63273
:10037000D107C9F70E942D200C9409260C94000087
:1003800080910008909101088737974709F0A89558
:100390000895DC01ED91FC910190F081E02D09952B
:1003A000089520919C0330919D03382748E0C901AE
:1003B000880F991F37FF06C09C0151E2252750E1A5
:1003C000352701C09C01415091F730939D03209344
:1003D0009C03089588E380939E0380E092ECA1E063
:1003E000B0E080939F039093A003A093A103B093E8
:1003F000A20387E08093AB0380EC92E9ADEEB9E114
:100400008093A3039093A403A093A503B093A603A2
:1004100085E08093AC038DEE9EEFADEABEED809358
:10042000A7039093A803A093A903B093AA03EDEAAE
:10043000F3E080E090E0863028F4DC01AC5DBD4F55
:100440002C9101C020E0219301968831910599F704
:1004500082E08093C5038AE08093C603089580EC10
:1004600091EDA8E9BBE18093E3039093E403A093AB
:10047000E503B093E60380E090E0A0E0B0E5809370
:10048000E7039093E803A093E903B093EA03EBEE4C
:10049000F3E080E081938F5F8031E1F70895A0E081
:1004A000B0E0E5E5F2E00C944725D82F0E943D1A14
:1004B0006115710581059105C9F30E94EA25109225
:1004C000A7031092A8031092A9031092AA03C4E0F4
:1004D000812C912C54018A94C090A703D090A8033A
:1004E000E090A903F090AA03FE2CED2CDC2CCC2488
:1004F0000E94E525A50194010E9426256C0D7D1D15
:100500008E1D9F1D6093A7037093A8038093A9037A
:100510009093AA03C15001F7DD2309F450C00DEAFE
:1005200013E0E801A12CB12C62E3C62ED12CE12C02
:10053000F12C8881882309F442C0B39419F40E94F5
:10054000EA013DC00E94E525A70196010E942625EB
:10055000E1E0E60FADEAB3E08A2F801B8A1520F4B4
:100560008D918E13F9CFE9CF2091AC0330E0A0E15B
:10057000B7E20E94BE249B01AC01AE2FB0E00E9406
:10058000CD244090A3035090A4036090A5037090E5
:10059000A603640D751D861D971D4090E3035090C2
:1005A000E4036090E5037090E6034616570668067C
:1005B000790618F2E993A39488E1A812BACFCDB7CF
:1005C000DEB7E0E10C94632580919B03813019F440
:1005D00082E080939B0380919B03833019F484E035
:1005E00080939B03089588E08093C10061E08AE0D6
:1005F0000E94151B60E08AE00E944E1B0895009740
:10060000C9F09C0140E050E068E478EE81E090E0C1
:100610000E9426252F3F31054105510529F020F084
:100620002FEF30E040E050E02093D1008091C000F7
:10063000806103C08091C0008F7E8093C0000895C8
:10064000219A229A239860E08BE00E94151B61E0BA
:100650008CE00E94151B0895EBE6F0E08081806835
:100660008083E8E6F0E080818160808308951F92B6
:100670000F920FB60F9211242F933F934F935F93D6
:100680006F937F938F939F93AF93BF93EF93FF935A
:100690001F9B0E94E402FF91EF91BF91AF919F9148
:1006A0008F917F916F915F914F913F912F910F901B
:1006B0000FBE0F901F901895A1E0B0E0E2E6F3E0C6
:1006C0000C9454251FB791E090939A03F894898372
:1006D0000E94C00198E1909360008981809360003E
:1006E00081110E94C0011FBF2196E3E00C94702588
:1006F0008F929F92AF92BF92CF92DF92EF92FF9232
:10070000CF93FC01C0A5EC2FE770F0E0E45EFD4F55
:10071000A081B0E0C7FF03C024E130E002C02FE0B9
:1007200030E0FC0197A183E1989FF0011124E25C85
:10073000FE4F80809180A280B380A20FB31F20E47F
:100740003FE14DE750E00E94D824A50194010E94AA
:1007500004258C2F887149F469017A01E0EDCE0EF1
:10076000E7E0DE1EE11CF11C1BC0C7FF05C060E412
:100770007AE88CE29EE004C060E07EEE8AEB9BE0CB
:1007800069017A01F8EBCF0EFBE0DF1EE11CF11CE2
:10079000A50194010E940425C20ED31EE41EF51E7D
:1007A000C701B60169517C4F8F4F9F4F28EE33E050
:1007B00040E050E00E940425A8EEB3E00E94CD2462
:1007C000CF91FF90EF90DF90CF90BF90AF909F9030
:1007D0008F9008958F3F910551F048F0811522E0E8
:1007E000920738F08115934030F482E0089580E05C
:1007F000089581E0089583E00895A0E0B0E0E3E08B
:10080000F4E00C945025EB018A01B82FB695A0E0D6
:1008100028813981F80120832A813B8121832C8121
:100820003D8122832E813F812383688179814A81A2
:100830005B812C813D81EE81FF819F2F9295990FE5
:10084000990F907C272F2370922B252F2370220F36
:10085000220F922B232F23702295207F922BF801B9
:1008600094830B5F1F4F2896AF5FBA1788F680FFFF
:1008700024C0888199810E94EA03D82E8A819B81B5
:100880000E94EA03E82E8C819D810E94EA03F82EE3
:100890008E819F810E94EA03F0E4DF9EA001112473
:1008A00090E1E99E90011124242B282BE4E0FE9E88
:1008B000B0011124262BF8012083CDB7DEB7E7E085
:1008C0000C946C25803223E0920708F1883E23E0E7
:1008D000920740F48F519340E4E096958795EA950E
:1008E000E1F70895803D27E0920718F48C5D93406E
:1008F0000895883928E0920768F4885C974074E08E
:10090000969587957A95E1F78D509C4F089580E0F4
:1009100090E008958FEF93E008958C30910540F4B6
:10092000A4E0880F991FAA95E1F7885D9C4F089570
:10093000843F23E0920718F484529C4F0895811558
:1009400024E0920740F48657934FF4E0880F991FF4
:10095000FA95E1F7089580E998E008959C013695AD
:10096000279525753575821B930B9C012373337373
:10097000969587959695879583739373820F931FAA
:100980009C0154E0369527955A95E1F7280F391FB9
:100990002F703F7041E051E0249FC001259F900DD2
:1009A000349F900D1124892F08952998882319F0D8
:1009B00000002A9A02C000002A980000299A00002C
:1009C0000895299A000083B12998000083FB8827A5
:1009D00080F90895CF93DF93D82F5E9A29985E9877
:1009E000C8E08D2F80780E94D504DD0FC150C9F773
:1009F0002998DF91CF9108958F770E94EA04089596
:100A0000CF93DF93D82FC8E08D2F80780E94D50434
:100A1000DD0FC150C9F72998DF91CF910895CF9389
:100A2000DF932998C8E080E0D82FDD0F0E94E10411
:100A30008D0FC150C9F7DF91CF9108950E94FC043A
:100A40000E940F055E9A0895A1E0B0E0EAE2F5E0A9
:100A50000C945525806869830E94EA046981862F79
:100A60000E9400055E9A2196E2E00C947125CF93D6
:100A7000C091A703C827E82FF0E0E256FC4F678536
:100A800089E70E9424056C2F8DE30E9424056C2FBA
:100A900082E40E942405CF91089586E20E941E05FB
:100AA0000895CF93DF93EC016C818CE10E942405C3
:100AB0006D818DE10E9424056E818EE10E942405E6
:100AC0006F8180E20E942405688581E20E942405EE
:100AD000698582E20E9424056A8583E20E942405DA
:100AE0006B8584E20E9424056C8585E20E942405C2
:100AF0006D858AE20E9424056E858EE60E9424059B
:100B00006F858FE60E942405688980E70E9424058E
:100B1000698981E70E9424056A8982E70E94240589
:100B2000DF91CF910895CF92DF92EF92FF92CF9312
:100B3000DF936B017C01C11488E3D8068CE9E806D9
:100B40008CE1F80628F5C701B60120E836E948E946
:100B500050E00E940425E901689760E879E687E69D
:100B60009FEF0E94E0246C0D7D1D8E1D9F1DF2E005
:100B7000660F771F881F991FFA95D1F721E732E09A
:100B800040E050E00E940425F22EE32E80E421C0D4
:100B9000C701B60120E03DE241E351E00E94042597
:100BA000E901689760E073ED8EEC9EEF0E94E0240F
:100BB0006C0D7D1D8E1D9F1D660F771F881F991F51
:100BC00021E732E040E050E00E940425F22EE32EBF
:100BD00080E66C2F6F71680F85E70E9424056E2DEB
:100BE00086E70E9424056F2D87E70E942405DF9188
:100BF000CF91FF90EF90DF90CF900895682F8DE612
:100C00000E94240508958F929F92AF92BF92CF9237
:100C1000DF92EF92FF92CF93DF93D82F83E00E9471
:100C20001E058093990384E00E941E05809398031B
:100C300060E086E00E94240561E087E00E942405D0
:100C40006FE789E00E94240565E08AE00E942405A0
:100C500065E18BE00E94240562E18CE00E9424059E
:100C60006DEF8DE00E94240560E08EE00E94240577
:100C7000DD2319F08BE291E008C02091C50333E138
:100C8000239FC0011124825C9E4F0E9451056CE895
:100C900080E30E9424056FE082E30E94240562E461
:100CA00083E30E9424058091C60387FF02C064E1AC
:100CB00001C06AE084E30E9424056AE285E30E94A1
:100CC00024056DE286E30E94240564ED87E30E941B
:100CD000240560E088E30E94240560E089E30E9427
:100CE0002405D11109C0C090A703D090A803E090BB
:100CF000A903F090AA0307C0C5E9CC2EC1ECDC2EF5
:100D0000ED2CCEEDFC2ECAE38F2C9924AA24BB2413
:100D1000682D8C2F0E942405682D85E08C0F0E9481
:100D20002405FE2CED2CDC2CCC24CF5FCE3361F7D8
:100D30006FEF83E40E9424056FEF84E40E94240592
:100D40006FEF85E40E9424056FEF86E40E9424057E
:100D5000DD2311F066E002C06091AB038DE60E94D6
:100D6000240560E089E70E9424056091AC038AE7CE
:100D70000E94240560E083E70E94240560E084E788
:100D80000E942405D11109C06091A3037091A403AE
:100D90008091A5039091A60304C060EC72E98DEEEA
:100DA00099E10E949305DF91CF91FF90EF90DF9042
:100DB000CF90BF90AF909F908F90089561E087E0B3
:100DC0000E94240564E28EE70E94240563E088E027
:100DD0000E94240560E088E00E94240565E087E029
:100DE0000E94240562E085E00E94240583E00E94C1
:100DF0001E058093990384E00E941E05809398034A
:100E0000089583E00E941E058093990384E00E9468
:100E10001E058093980361E087E00E9424056AE044
:100E200070E080E090E00E94601A0E94DE06000000
:100E30000895CF92DF92FF920F931F93CF93DF938A
:100E40001F92CDB7DEB7082F162F8EE399830E942D
:100E50002405F02EC02E9981D92E8C2D8F19811743
:100E600038F4F60161916F018FE70E942405F5CFF8
:100E700064E085E00E94240583E00E941E058093C3
:100E8000990384E00E941E05809398030E943D1AF6
:100E900060939403709395038093960390939703C4
:100EA00069E087E00E94240581E080939B030F9016
:100EB000DF91CF911F910F91FF90DF90CF90089518
:100EC0000F931F930E94190780919B03813099F41F
:100ED0000E943D1A0091940310919503209196036E
:100EE00030919703601B710B820B930B603A76482D
:100EF0008140910548F380919B03813031F467EA8A
:100F000071E086E094E00E94451D1F910F910895C5
:100F10000F931F9380919B03823021F410929B03C7
:100F200081E020C080919B038130D9F40E943D1A5A
:100F300000919403109195032091960330919703AB
:100F4000601B710B820B930B613A764881409105CF
:100F500040F061E087E00E94240510929B0382E04C
:100F600001C080E01F910F910895CF93DF93EC01B2
:100F70004AE050E06D2F70E086E094E00E940A1E87
:100F80006EE286E094E00E94171DBE0184E0769533
:100F900067958A95E1F76F7077274AE050E086E021
:100FA00094E00E940A1E6EE286E094E00E94171D03
:100FB000BE016F7077274AE050E086E094E00E941F
:100FC0000A1EDF91CF910895D82FC0E0CD1780F48D
:100FD0005F9A64E670E080E090E00E94601A5F989B
:100FE00064E670E080E090E00E94601ACF5FEECF90
:100FF0006CE271E080E090E00E94601AE6CF0F930F
:101000001F93CF93DF93EC01062F15E0115051F0A1
:10101000CE010E94F325081741F0602FCE010E94F7
:10102000FB25F4CF82E00E94E407DF91CF911F916E
:101030000F910895A0E0B0E0E0E2F8E00C944725BD
:10104000482E562EC0E0D0E0612C712CE12CF12C02
:1010500000E010E041100CC06090FC0386E4689E44
:101060003001112459E1E52EF12C02EE13E01EC0EF
:1010700091E049120FC06090FC03E6E46E9E3001DF
:101080001124FBE16F0E711C49E2E42EF12C0EE9F4
:1010900013E00CC082E0481209C028E1622E7724D8
:1010A0007394EE24E394F12C0BEF13E043018C0EC8
:1010B0009D1E10929D0310929C033401A62CA8182B
:1010C000B12CC30101966C01AE14BF04A8F4A00EAC
:1010D000B11E511006C0C3010E94F325F5018083A3
:1010E00005C0F5016081C3010E94FF07F501808101
:1010F0000E94D1013601E2CFC301511018C0C301D3
:101100000E94F325B82EC6010E94F3252B2D30E056
:10111000322F2227282B80919C0390919D038217C8
:10112000930779F4C0E0D0E05524539493CF36016F
:1011300060919D030E94FF0760919C03C6010E947D
:10114000FF07C05EDE4FC13E92E0D90708F482CFB0
:10115000852DCDB7DEB7E0E10C94632561E082E038
:101160000E941A08089560E082E00E941A088091A7
:10117000FB03853020F01092FB030E94AE088091A3
:10118000FB038093FC03089561E080E00E941A084D
:1011900061E081E00E941A08089560E080E00E940A
:1011A0001A08882351F060E081E00E941A08882321
:1011B00021F080919E03883349F00E942F020E9403
:1011C000EA0181E00E944F020E94C4080895CF9373
:1011D000C82F0E943D1A609358037093590380935F
:1011E0005A0390935B03C0936D03CC2329F040E036
:1011F00051EE60E070E004C040E855E260E070E06D
:1012000088E594E00E94701FCF91089590915C034F
:10121000492F4F7050E0BA016F5F7F4F292F30E0A8
:10122000E4E035952795EA95E1F76217730759F0E1
:10123000FA01E35AFC4F808381E0890F8F70907F21
:10124000892B80935C0308956EE770E088E594E055
:101250000E94C9010895A3E1B1E0E1E3F9E00C9433
:101260004825EDEAF3E0712C8191882321F07394F5
:1012700028E17212F9CF63EB71E086E094E00E94FE
:10128000451D4AE050E0672D86E094E00E94111E63
:1012900080E00E9403060E94DE068E010E5F1F4F53
:1012A000C12CD12C7601C39466246A945C2C0E94D4
:1012B000311A4B015C012091AC0330E0A0E1B7E2B0
:1012C0000E94BE249B01AC01C701B6010E94E0242C
:1012D0002091A3033091A4034091A5035091A6034C
:1012E000620F731F841F951F2091E3033091E40365
:1012F0004091E5035091E603261737074807590741
:1013000018F4F801608225C08C2D0E94370561E039
:1013100070E080E090E00E94601AF80110820E9464
:10132000311A681979098A099B09643F714081055E
:10133000910540F40E944D05F8019081981778F7C7
:101340008083EDCF50FE03C046985F9A02C0469A54
:101350005F982FEFC21AD20AE20AF20A0F5F1F4FFC
:101360008FEFC816D104E104F10409F09FCFCE013C
:101370009395FC01D82E7FEF68EC2E2F281B2715A4
:1013800010F051E056C0DE01129651E02FEF41E01F
:101390003D91321710F0322F01C0452F5F5F5F3F44
:1013A00011F0232FF5CF4193242F30E0A1E0B0E0DE
:1013B000AC0FBD1FA20FB31F5C93413079F0DE016B
:1013C000A20FB31F5C93423049F0AFEFBFEFAC0FF9
:1013D000BD1FA20FB31F6C934E3F78F6A2E0B0E0A2
:1013E000AC0FBD1FA20FB31F7C934D3F30F6A3E09F
:1013F000B0E0AC0FBD1FA20FB31F6C93BECF452F43
:10140000242F30E0FC01E20FF31F6081AFEFB0E06A
:10141000AC0FBD1FA20FB31F2C91621748F44150AF
:10142000DC01A40FB11D2C9120836C934111E8CFF6
:101430005F5F571520F3372D369520E0231770F4A2
:10144000DC01A20FB11D4C91522F530FFC01E50F8F
:10145000F11D50815C9340832E5FF0CFFDEAEF2EAB
:10146000F3E0FF2E8C01802F8D19871598F4F80179
:10147000C1908F014AE050E06C2D86E094E00E941C
:10148000021E6CE286E094E00E94171DF701C192F3
:101490007F01E9CF86E094E00E941F1D81E0CD5ED0
:1014A000DE4FEFE00C9464251F920F920FB60F925F
:1014B00011241F932F933F934F935F936F937F93C9
:1014C0008F939F93AF93BF93CF93DF93EF93FF934C
:1014D000C0918600D09187008091170390911803E6
:1014E00020913903211155C09E01281B390B809191
:1014F000E7039091E803A091E903B091EA0385FD29
:1015000002C036952795253C49E03407B8F1409153
:101510000A0150E060E070E02CE1B695A795979540
:1015200087952A95D1F70097A105B10521F481E0AF
:1015300090E0A0E0B0E084179507A607B707D8F4BD
:1015400080910A018F3FB9F040E080910A0148176D
:1015500080F4842F90E0880F991FFC01E75EFC4F18
:1015600020813181FC01E55FFE4F318320834F5F95
:10157000ECCF10923A0310920A010BC02D3B82E08F
:10158000380720F080910A018031D8F08FEF8093E6
:101590000A01D0931803C0931703FF91EF91DF91D5
:1015A000CF91BF91AF919F918F917F916F915F91FB
:1015B0004F913F912F911F910F900FBE0F901F9051
:1015C000189510910A0181E0810F80930A01C901E9
:1015D0000E946204E12FF0E0EE0FFF1FE75EFC4F78
:1015E00091838083D6CF83E0809380008AE98093C3
:1015F00081008091E70386FD05C0809181008064B1
:10160000809381008FEF9FEF9093890080938800F3
:1016100080916F00806280936F0008950E94B308EC
:101620008091FC03843011F41092FC0308956F3014
:1016300018F086958058089589E0689F802D1124C0
:101640000895A0E0B0E0E7E2FBE00C944F25C82F3E
:101650000E943D1A0091C8021091C9022091CA024D
:101660003091CB026B017C01C01AD10AE20AF30A65
:101670009701860149E8C41643E1D406E104F10468
:1016800010F01092CC026093C8027093C90280934C
:10169000CA029093CB02209139038FEF820F8230E0
:1016A000D8F5E091CC02EE2309F44EC1E13011F4FB
:1016B00082E0B8C1E03108F034C181E08E0F809340
:1016C000CC02F0E0E75EFC4FC083803109F0ACC192
:1016D000EBE1F3E0213029F4A181A695A695808164
:1016E00008C080819181A92FA695A695A69596956B
:1016F0008795A03148F4B0E090E0AA0FBB1FA55F2A
:10170000BE4F11969C938E9310923A03329683E0CB
:10171000E932F807F9F688C1233009F005C1E091F4
:10172000CC02E11104C0CF3009F07EC10DC1E83117
:1017300048F481E08E0F8093CC02F0E0E85EFC4F2D
:10174000C08372C1E83109F0ECC0C111EAC040E0C9
:1017500050E0ABE0CA01B3E0880F991FBA95E1F7FA
:10176000A49F9001A59F300D1124F901E75EFC4F65
:101770006081E1817E2F777075956795FC01EE0F92
:10178000FF1FE55FFE4F71836083F901E65EFC4F4A
:10179000B081B695B695B695E181FE2FF295FF0F13
:1017A000F07E6F2F6B2BE695E695E6957E2F777092
:1017B00075956795FC01EE0FFF1FE35FFE4F718388
:1017C0006083F901E55EFC4FB081B295B695B695A0
:1017D000B370C181DC2FDD0FDD0F6D2F6B2BC29538
:1017E000C695C695C370E281E170EE0FEE0F7E2FB5
:1017F0007C2B75956795FC01EE0FFF1FE15FFE4F97
:1018000071836083F901E35EFC4FB081B695E1819D
:10181000FE2FF795FF27F7956F2F6B2BE6957E2F01
:10182000777075956795FC01EE0FFF1FEF5EFE4F19
:1018300071836083F901E25EFC4FB081B295BF70A5
:10184000E181FE2FF295F07F6F2F6B2BE295EF7009
:101850007E2F777075956795FC01EE0FFF1FED5E8B
:10186000FE4F71836083F901E15EFC4FB081BB1FC5
:10187000BB27BB1FC181DC2FDD0F6D2F6B2BCC1F56
:10188000CC27CC1FE281E370EE0F7E2F7C2B759569
:101890006795FC01EE0FFF1FEB5EFE4F71836083C7
:1018A000F901EF5DFC4FB081B695B695E181FE2F51
:1018B000F295FF0FFF0FF07C6F2F6B2BE695E695EF
:1018C0007E2F777075956795FC01EE0FFF1FE95E1F
:1018D000FE4F71836083F901EE5DFC4F20812295FC
:1018E000269527703181E32FEE0FEE0FEE0F6E2F4E
:1018F000622B732F72957695777075956795FC01BD
:10190000EE0FFF1FE75EFE4F718360834F5F5F4FF7
:101910004230510509F01ECF80912F0383FF1092B2
:101920003A031092CC0280C0243009F07DC060914F
:10193000CC0261110BC0C83AB1F410929D03109211
:101940009C0388EA0E94D10181E06CC0613019F4E7
:10195000C093C70204C0623031F4C093C6028C2F1A
:101960000E94D1015AC0E091C6022E2F30E0220F12
:10197000331F462F50E0C9010296841795073CF0AB
:10198000633268F7FA01EA5EFC4FC083E8CF2D5F4F
:101990003F4F8C2F90E060919C0370919D03421704
:1019A000530749F4982F88278627972790939D03FC
:1019B00080939C0332C06817790769F58091C7024C
:1019C000813049F5E13118F080E18093C602F09052
:1019D000C602CAE1D3E000E010E00F15D0F4FE012A
:1019E0003197808190E0982F88272881822B63E0AF
:1019F000969587956A95E1F70E946204F801EE0FCB
:101A0000FF1FE55FFE4F918380830F5F1F4F22967C
:101A1000E4CF10923A031092CC028091CC0288233A
:101A200019F08F5F8093CC02CDB7DEB7E8E00C945D
:101A30006B25E82FF0E0EE51FC4FE185E03150F4EA
:101A4000F894F0E0EE0FFF1FE55FFE4F808191817B
:101A500078940895E03121F0E13169F483E001C028
:101A600082E00E94811B892B19F084EF93E0089596
:101A70008CE090E0089580E092E00895A2E2B0E06A
:101A8000E4E4FDE00C9445259E012F5F3F4F80E18B
:101A9000D9011D928A95E9F761EE71E086E094E044
:101AA00029A33AA30E94451D0E9401071D8A1E8A90
:101AB0001F8A188E312C212C00E0812C912C54018E
:101AC00070E4472E71EE572E7DE9672E78E1772E70
:101AD000E0E5CE2EE3ECDE2EE12CF12C84EF91E05C
:101AE000A0E0B0E08D8F9E8FAF8FB8A380EC91ED1A
:101AF000A8E9BBE1898F9A8FAB8FBC8F80E491EE10
:101B0000ADE9B8E1898B9A8BAB8BBC8B86E094E016
:101B10000E94AA1B892B09F4E1C086E094E00E9490
:101B2000CE1B9C0133272C32310509F442C0ACF4A2
:101B30002332310509F0ABC019821A821B821C8244
:101B40001D821E821F82188619861A861B861C8695
:101B50001D861E861F86188A60C02434310529F030
:101B60002335310509F4B2C092C064E486E094E004
:101B70000E94171D2AE030E040E451EE6DE978E163
:101B800086E094E00E94A51D6CE286E094E00E944D
:101B9000171D2AE030E040EC51ED68E97BE186E07A
:101BA00094E00E94A51D6CE286E094E00E94571D1F
:101BB000ADCF0F5F043009F0A9CF29813A814B8165
:101BC0005C81A8EEB3E00E94CD24698B7A8B8B8B6D
:101BD0009C8B2D813E814F8158850E94CD24698F39
:101BE0007A8F8B8F9C8F29853A854B855C852D8FCD
:101BF0003E8F4F8F58A32D853E854F8558890E9473
:101C0000CD246B017C0160323EE4730781059105B0
:101C100030F462E38CE10E94240500E077CF60336A
:101C200045E774078105910510F462E2F3CF603453
:101C30005CE975078105910510F466E2EBCF80E55C
:101C4000C81683ECD806E104F10410F462E1E2CF97
:101C500090E6C9169AEED906E104F10410F465E1A4
:101C6000D9CFA0E7CA16A1E1DA06A1E0EA06F1049D
:101C700010F461E0CFCFB0EACB16B6E8DB06B1E0F6
:101C8000EB06F10410F463E0C5CF65E0C3CF10EDBF
:101C9000180F1A3008F03ACFE1E0F0E0EC0FFD1F2A
:101CA00024E0029FE00DF11D112420813181428149
:101CB0005381AAE0B0E00E94CD24610F711D811D07
:101CC000911D608371838283938320CF49885A88D2
:101CD0006B887C88812C912C540118CF811491043D
:101CE000A104B10489F4C301B2010E94930561E02B
:101CF00070E080E090E00E94601A1D8A1E8A1F8AB0
:101D0000188E312C22242A948D8D9E8DAF8DB8A1F2
:101D100088169906AA06BB06D0F40E944D052D89A7
:101D20003E894F89588D280F311D411D511D2D8B26
:101D30003E8B4F8B588F381608F4382E821508F4D6
:101D4000282E3FEF831A930AA30AB30A56C0C30191
:101D5000B20128EE33E040E050E00E940425BA01D1
:101D6000A9012AE030E086E094E00E94F31D6CE2D5
:101D700086E094E00E94171D4AE050E0632D86E063
:101D800094E00E94021E6CE286E094E00E94171D1F
:101D90006D897E898F89988DA50194010E94042503
:101DA000BA01A9012AE030E086E094E00E94F31D28
:101DB0006CE286E094E00E94171D4AE050E0622D3C
:101DC00086E094E00E94021E6CE286E094E00E94AD
:101DD000571D4C0C5D1C6E1C7F1C898D9A8DAB8D24
:101DE000BC8D84159505A605B70520F449885A8849
:101DF0006B887C88812C912C540129893A894B89E4
:101E00005C89283E33404105510509F07FCEA296FA
:101E1000E2E10C946125ACE1B0E0E1E1FFE00C947B
:101E20004F250E943D1A6B017C0181E00E94030650
:101E300014E703E0198361E0CE0101960E94600778
:101E400000939B030E94DE066AEF70E080E090E062
:101E50000E94601A80919B03833089F486E094E0AD
:101E60000E94AA1B892B59F40E943D1A6C197D0906
:101E70008E099F096038734C894C9140D8F280914B
:101E80009B03833009F44FC08FE70E94FC040E943B
:101E90000F058983843511F083E05CC00E940F0533
:101EA00010926E0380936F030E940F0520916E03C2
:101EB00030916F03280F311D30936F0320936E0311
:101EC0000E940F05809370030E940F058093710399
:101ED000813110F7F12C0F2D10E08091710390E00B
:101EE000880F991F0817190740F40E940F05F80181
:101EF000EE58FC4F8083F394EECF80E7898361E056
:101F0000CE0101960E94600783E080939B030E94AC
:101F1000DE0662E370E080E090E00E94601A80914B
:101F20009B03833011F482E015C08FE70E94FC040C
:101F30000E940F058983803509F0AECF07EC13E0CE
:101F40000E940F05F80181938F01F3E0023E1F0705
:101F5000B9F781E06C96E8E00C946B25CF93C82F1D
:101F6000682F86E094E00E941B1C909192039C27AE
:101F700090939203CF910895A1E0B0E0E2ECFFE0EE
:101F80000C94552599830E94AE0F9981892F0E9448
:101F9000AE0F2196E2E00C9471251F93CF93DF934F
:101FA000182FEB011092920365EB86E094E00E94FB
:101FB0001B1C62E686E094E00E941B1C812F0E949D
:101FC000AE0FCE010E94BC0FDF91CF911F910895FB
:101FD0006091920386E094E00E941B1C0895A1E2A8
:101FE000B0E0E5EFFFE00C9451257B018A018C30D5
:101FF00009F452C108F040C0863009F4BCC018F59D
:10200000833009F491C070F4813009F472C08230D9
:1020100009F047C26BE170E082E00E94CD0F07EC4F
:1020200013E078C0843009F487C0853009F039C2E4
:102030006091710370E0660F771F85E00E94CD0FFD
:1020400002E713E086C0893009F4A7C070F4873036
:1020500009F49BC0883009F024C261E070E088E098
:102060000E94CD0F8091FC0322C28A3009F4CAC0BD
:102070008B3009F4F1C015C28A3609F474C1D8F462
:10208000873609F439C138F4853609F40DC186362E
:1020900009F41EC106C2883609F436C1893609F032
:1020A00000C261E070E089E60E94CD0F0E94EA0163
:1020B0000E942F02F4C18D3609F4D3C138F48B3657
:1020C00009F490C18C3609F499C1EBC18E3609F43C
:1020D000DBC1873C09F0E5C161E070E087EC0E945C
:1020E000CD0F81E00E94AE0F0E94E80F1092930383
:1020F000E2C169E270E081E00E94CD0F0EE913E0D9
:10210000F80181918F010E94AE0FF3E0073C1F0799
:10211000B9F7CFC1F80181918F010E94AE0FF3E0B2
:10212000023E1F07B9F7C5C161E070E083E00E947D
:10213000CD0F0E940B0FBBC161E070E084E00E94F4
:10214000CD0F81E00E94AE0F0E94E80F0E943E0D6D
:10215000B2C18091710390E0880F991F98012257B6
:1021600033402817390708F0A4C1F80181918F0185
:102170000E94AE0FEECF62E070E086E00E94CD0FCD
:1021800081E893E00E94BC0F94C161E070E087E0B9
:102190000E94CD0F809170038AC186E6898361E039
:1021A000CE0101960E9460070E94DE0683E08093C4
:1021B0009B0368EC70E080E090E00E94601A8091E0
:1021C0009B038430D9F48FE70E94FC040E940F0522
:1021D0008983863469F460E270E089E00E94CD0F63
:1021E00010E20E940F050E94AE0F1150D1F761C19D
:1021F00061E070E089E00E94CD0F51C161E070E0C4
:1022000089E052C169E170E08AE00E94CD0F10922E
:10221000E20320919A038091E7039091E803A09153
:10222000E903B091EA03222311F0806801C08F779F
:102230008093E7039093E803A093E903B093EA0344
:1022400002EE13E0F80181918F010E94AE0FF3E0DE
:102250000B3F1F07B9F72DC161E270E08BE00E94D0
:10226000CD0F80913A038F3F39F080913A0391E08E
:10227000980F90933A0302C080913A030E94AE0FE8
:1022800010E0812F0E94190D0E948D040E94BC0F46
:102290001F5F1031B1F70DC161E070E08CE00E946A
:1022A000CD0F8091FB0303C161E070E085E60E94E1
:1022B000CD0F89E2E816F10409F0F8C0D801EEE983
:1022C000F3E08D91819383E0E73CF807D1F7E7C015
:1022D00061E070E086E60E94CD0FEBE1EE16F104BE
:1022E00009F0E4C0D801E7ECF3E08D91819383E03D
:1022F000E23EF807D1F7D3C061E070E087E60E94C4
:10230000CD0F0E94C408CBC061E070E088E60E9457
:10231000CD0F85E789838BE1E7ECF3E0DE011296D0
:1023200001900D928A95E1F76CE1CE0101960E9431
:1023300060070E94DE0683E080939B0360E273E007
:1023400080E090E00E94601A80919B03843009F045
:10235000ADC08FE70E94FC040E940F05898385357C
:1023600009F0A4C09CC061E070E08AE60E94CD0F35
:1023700089E6898361E0CE0101960E9460070E9490
:10238000DE0683E080939B0360E273E080E090E0F0
:102390000E94601A80919B03843009F087C08FE708
:1023A0000E94FC040E940F0589838E010E5F1F4F5F
:1023B0007E01EDE1EE0EF11C0E940F05F801819304
:1023C0008F01EE15FF05C1F78BE1FE013296A7ECF8
:1023D000B3E001900D928A95E1F78981893409F083
:1023E00065C05DC061E070E08BE60E94CD0FF80132
:1023F00080818093FC030E94CD0851C061E070E0B1
:102400008CE60E94CD0FF0E2EF16F10461F487E64E
:10241000898380E2F801DE01129601900D928A957F
:10242000E1F761E203C087E4898361E0CE010196B0
:102430000E9460070E94DE0683E080939B036CE4A9
:1024400074E080E090E00E94601A80919B038430E9
:1024500069F58FE70E94FC040E940F05873431F56F
:102460001EC061E070E08DE60E94CD0F89E1E816A4
:10247000F104E1F4D801E2EEF3E08D91819383E081
:10248000EB3FF807D1F70BC061E070E08EE60E94E9
:10249000CD0FF80180818093FB030E94AE0881E09C
:1024A00006C061E070E08AEC0E94CD0F80E00E94DF
:1024B000AE0F0E94E80FA196E6E00C946D25A0E017
:1024C000B0E0E5E6F2E10C944F25CAE5D2E014E66F
:1024D00006E035E0F32E44E0E42E53E0D52E62E032
:1024E000C62E86E094E00E94AA1B892B09F49BC0AB
:1024F00086E094E00E94CE1B282F8093C502409175
:10250000C40250E04730510560F7FA01EA5AFF4F24
:102510000C947C25853B29F781E08093C402E1CFB0
:10252000823609F07DC0C092C402DBCF8093C30223
:102530008093C202D092C402D4CF9C01332730933F
:10254000C1022093C0029091C20298279093C202C8
:10255000E092C402C6CF382F22274091C00250918A
:10256000C102242B352B3093C1022093C0029091DD
:10257000C20298279093C202F092C4022536310518
:1025800008F4AFCF61E070E08CEC0E94CD0F81E0E9
:102590000E94AE0F0E94E80F43C02091BE0230910E
:1025A000BF02F901E65AFD4F80839091C20298273D
:1025B0009093C202C90101969093BF028093BE021C
:1025C0002091C0023091C1028217930708F489CF8D
:1025D0000093C40286CF8091C20282130BC0609127
:1025E000BE027091BF024AE552E08091C3020E9490
:1025F000EF0F0DC062E070E08BEC0E94CD0F809178
:10260000C3020E94AE0F809192030E94AE0FFE01A2
:10261000812F11928A95E9F71092BF021092BE02A3
:102620001092C4025ECFCDB7DEB7E8E00C946B2504
:1026300081E08093930380919303882349F086E09F
:1026400094E00E94AA1B892BB1F30E945F12F3CF82
:102650000895AAE2B0E0EFE2F3E10C944D250E9468
:10266000311A6B017C0181E00E94030686E094E050
:102670000E94AA1B892B29F086E094E00E94CE1BC1
:10268000F5CF5F9811E072E6B72EE9E2AE2E03E0D7
:102690000E94311A6C197D098E099F09693C7105E8
:1026A00081059105D0F11123C1F10E94311A6B010E
:1026B0007C01469A80ED97E00E94FF02B982EEE924
:1026C000F3E0DE0112968A2D01900D928A95E1F7D2
:1026D0006AE2CE0101960E946007469880E090E091
:1026E0000E94FF0200939B030E94DE0662E370E0FB
:1026F00080E090E00E94601A80919B03843061F436
:1027000000939B038FE70E94FC040E940F0511E0D9
:10271000823419F410E001C011E082E10E94811BB3
:10272000892B81F411E00EC05F9A469A86E094E00E
:102730000E94CE1B8D309105A9F05CF40A9791F0B0
:102740005F98469886E094E00E94AA1B892B61F767
:102750009FCF8332910569F08234910589F70E94F9
:102760001813EECF66ED70E086E094E00E94331D12
:10277000E7CF0E943E0DE4CF8F929F92AF92BF921F
:10278000CF92DF92EF92FF921F93CF93DF9382E17C
:102790000E94811B892B09F089C068EC70E080E001
:1027A00090E00E94601A80E090E00E94FF020E9488
:1027B000311A4B015C016B017C0180ECC80E82E197
:1027C000D81EE11CF11C0E94311A6C157D058E0586
:1027D0009F0530F482E10E94811B892BA1F364C024
:1027E00082E10E94811B892B09F05EC080ED97E099
:1027F0000E94FF020E94311A6B017C01D0E0C1E00F
:1028000088E4880E86E2981EA11CB11C11E082E1CA
:102810000E94811B892B21F58C149D04AE04BF04FA
:1028200030F480ED97E00E94FF02D1E0F0CF0E94EB
:10283000311A6C197D098E099F09693C7105810562
:10284000910528F30E94311A6B017C01C12719F010
:1028500080ED97E002C080E090E00E94FF02D7CFB9
:1028600080E090E00E94FF02DD23B9F08091FB033D
:1028700090E0019665E070E00E94F0248093FB03F5
:102880000E94AE080E940E0B0E94CD0864EF71E01A
:1028900080E090E00E94601A09C080E00E944F0230
:1028A0000E942B090E94C4080E942913DF91CF9136
:1028B0001F91FF90EF90DF90CF90BF90AF909F90CF
:1028C0008F900895CF92DF92EF92FF9280E00E9466
:1028D0005C030E94200361E086E00E94151B61E01A
:1028E00085E00E94151B60E082E10E94151B60E0FC
:1028F00084E00E94151B61E084E00E944E1B0E9450
:10290000F30260E070E086E094E00E94A01C0E9468
:102910000E0B0E94CD080E94F30A8FEF80933A03BA
:102920000E942C0378940E94311A6B017C018091E3
:102930003A038F3F59F40E94311A6C197D098E09B0
:102940009F09603D77408105910588F380ED97E010
:102950000E94FF0261E082E10E944E1B5F9A86E0C6
:1029600094E00E94AA1B892B29F086E094E00E9443
:10297000CE1BF5CF6EEE71E086E094E00E94141D50
:1029800081E893E00E94B50765E072E086E094E09C
:102990000E94141D4AE050E066E070E086E094E09A
:1029A0000E94DB1D62E370E080E090E00E94601A0C
:1029B00086E094E00E94AA1B04970CF186E094E064
:1029C0000E94CE1B82349105D1F486E094E00E94EF
:1029D000CE1B8E34910599F486E094E00E94CE1BC4
:1029E0008434910561F486E094E00E94CE1B8197C7
:1029F00031F480E090E00E94FF020E942913409190
:102A00009F035091A0036091A1037091A203DB0189
:102A1000CA010197A109B1090497A105B10568F49C
:102A200040933903433029F440EA56E861E070E00E
:102A300004C040E052EC61E070E088E594E00E9460
:102A4000701F0E94BC135F9880E090E00E94FF021C
:102A50000E94F30A109255038091E70383FF11C08F
:102A60008091B303882351F08091BA03882331F019
:102A70008091C103882311F087E001C085E0809335
:102A8000550380E00E940306809156030E9437059B
:102A90000E94DE061092CF021092CE021092CD025A
:102AA000F12C8091FC038F15B0F062E370E080E0C0
:102AB00090E00E94601A80ED97E00E94FF0262E3BE
:102AC00070E080E090E00E94601A80E090E00E9458
:102AD000FF02F394E6CF8091C60384FF08C0982FCD
:102AE000987181E0983109F080E00E94E7088FE05A
:102AF0000E945C03FF90EF90DF90CF900895EF92DB
:102B0000FF920F931F93CF93DF938C016EE770E0DA
:102B100088E594E00E94C901E801F12CF0E2EF2E73
:102B20008E0188818D57823048F46DE770E088E52A
:102B300094E00E94C90188818E2588832196F8013E
:102B4000608188E594E00E94821EF394F9E0FF1210
:102B5000E7CF6EE770E088E594E00E94C901CDB749
:102B6000DEB7E6E00C946D25A9E0B0E0EAEBF5E114
:102B70000C9455259091570391110EC09EEF9983A7
:102B80008A836B8350E0559547954C832D83198636
:102B900018861F821E822EC040915C03842F90E015
:102BA000B4E095958795BA95E1F7242F2F7030E022
:102BB0008217930719F18DEF89831B82FE013496EA
:102BC00050E0842F90E0A4E095958795AA95E1F7D1
:102BD000242F2F7030E08217930749F0DC01A35AAD
:102BE000BC4F8C918193405F5F5F563051F74093AB
:102BF0005C035A83CE0101960E947F158091570392
:102C000090E0019666E070E00E94F0248093570304
:102C10002996E2E00C947125A0E0B0E0E2E1F6E153
:102C20000C944E256C016EE770E088E594E00E94FC
:102C3000C9018601E12CF12CC0E0D0E030E2B32ED6
:102C4000F801608183E8860F823078F46DE770E0E8
:102C500088E594E00E94C901F80160816B2570E06D
:102C600088E594E00E94C90104C088E594E00E94D0
:102C7000821EE114F10459F0F80180819E01280FB1
:102C8000311DC901C92FDD27C80FD91FDD273FEF2F
:102C9000E31AF30A89E0E816F10459F028E0E21695
:102CA000F10421F48C2F8095F60180870F5F1F4F70
:102CB000C7CFCDB7DEB7E9E00C946A25A9E0B0E054
:102CC000E4E6F6E10C945525E82F362F8091570362
:102CD00090E0019664E270E00E94F0248093570334
:102CE00058E9598350E15A83813089F048F08230A5
:102CF000B9F08330D9F48B8381EF8C833D8319C085
:102D000085E08B8381EF8C832F5F2D8312C08B83B3
:102D100081EF8C8384E6489FA00111245D8309C064
:102D200084E08B8381EF8C83ED8303C00E942409B0
:102D300004C0CE0101960E940C162996E2E00C9484
:102D40007125A2E0B0E0E7EAF6E10C944A25182FDD
:102D5000762E2A8349830E943D1A6B017C01809163
:102D60006D038090580390905903A0905A03B0903F
:102D70005B032A8149818823C1F0D701C6018819E4
:102D80009909AA09BB094C015D0191EE89169EE2E1
:102D90009906A104B10420F1241708F4422F202F32
:102DA000672D812F0E945E1613C0D701C6018819B6
:102DB0009909AA09BB094C015D0191E3891695E7C0
:102DC0009906A104B10460F0672D812F0E94B4150B
:102DD000C0925803D0925903E0925A03F0925B03D9
:102DE0002296EDE00C946625A2E2B0E0EAEFF6E16F
:102DF0000C944B258CE00E941E0581110DC06DE0E6
:102E000072E086E094E00E94451D5F9A80E00E9497
:102E100003060E94DE065F9888E594E00E94281E63
:102E2000892B01F188E594E00E94551E90913903A9
:102E3000992319F00E94210BEFCF4091CE0250E070
:102E40009A012F5F3F4F2F7133276091CF0270E0BF
:102E50002617370709F3FA01E752FD4F80832093C5
:102E6000CE02DACF80913903811106C080919B0395
:102E7000843009F094C00DC086E094E00E94AA1B43
:102E8000892BA1F386E094E00E94CE1B0E94210BC7
:102E9000F3CF0E943D1A611571058105910549F036
:102EA00060934703709348038093490390934A03C8
:102EB0000CC081E090E0A0E0B0E0809347039093E5
:102EC0004803A0934903B0934A0380913D03909136
:102ED0003E03816090933E0380933D0383E08093A3
:102EE0009B038FE70E94FC0409EF12E00E940F058C
:102EF000F80181938F01F3E002301F07B9F72091A9
:102F000002038091F902982F922796FF3BC090E42C
:102F1000922790930203982F98739833F1F410E05E
:102F2000212F30E08091F902877090E0821793079B
:102F30004CF11F5F2091C603812F90E0FC01E75008
:102F4000FD4F24FF04C080810E940609E9CF608103
:102F500088E594E00E94821EE3CF8F7399F48091FC
:102F6000FA02809346038091FB0280934403809190
:102F7000FC02809343038091FF0290E090933C0316
:102F800080933B038091CD02813019F482E08093DD
:102F9000CD028091CD02833011F41092CD020E94B7
:102FA0003D1A6B017C0180913F0390914003A091F9
:102FB0004103B09142030097A105B105C9F0A701F3
:102FC0009601281B390B4A0B5B0BDA01C901883BC0
:102FD0009B40A105B10560F00E944D05809345031B
:102FE00010923F031092400310924103109242034B
:102FF00080914B0390914C03A0914D03B0914E03EF
:1030000046015701881A990AAA0ABB0A8EE993E079
:103010000E94780386169706A806B90608F4A8C089
:10302000C0924B03D0924C03E0924D03F0924E03BA
:103030000E94C00180913A038830A0F08091E7039C
:103040009091E803A091E903B091EA036CE1B69591
:10305000A795979587956A95D1F7892B8A2B8B2B06
:1030600009F0A4C180913A038F5F80933A03809165
:10307000470390914803A0914903B0914A030097F8
:10308000A105B105F1F0C81AD90AEA0AFB0A8EE9CE
:1030900093E00E9478036C157D058E059F0508F06E
:1030A00006C18091E70384FD04C080ED97E00E9493
:1030B000FF021092470310924803109249031092A6
:1030C0004A0390910203907C909302035091CE02A8
:1030D0008091CF022091CD02581709F405C122300A
:1030E00009F002C1905890930203E091C603E77083
:1030F000F0E0E45EFD4F6081693008F0DDC06150B2
:1031000040E04613DBC08093CF0287E3840F9091A9
:103110000203892B809302034093D00283E08093C3
:10312000CD02469A8091AB039091550391112FC126
:103130000E94FE05809156030E943705E091C60368
:10314000E770F0E0E45EFD4F608182E093E00E9472
:103150001907E0915603EF5FE0935603E83109F455
:1031600022C1F0E0E256FC4F8785882309F41BC199
:103170000E948807813069F58091C603887149F102
:1031800080913D0390913E03880F991F90933E03D9
:1031900080933D0383E080939B030E94DE060E94A0
:1031A0003D1A60933F0370934003809341039093D3
:1031B0004203672B682B692B61F481E090E0A0E06B
:1031C000B0E080933F0390934003A0934103B093FA
:1031D00042038091C60384FF1FC080913D039091FC
:1031E0003E038E7F0E94AE04182F60913B038091B6
:1031F00046030E94170B482F612F8091450349A376
:103200000E94170B0091FC03282F49A160914303F2
:10321000809144030E94A116469880915303813007
:10322000C1F018F08230B1F1CEC082E10E94811B62
:10323000892B09F0C8C081E0809353030E94311AA2
:1032400060934F0370935003809351039093520304
:10325000BAC082E10E94811B892B31F50E94311A8C
:10326000C0904F03D0905003E0905103F090520370
:103270006C197D098E099F09693E7340810591058E
:1032800008F4A1C082E08093530380ED97E00E9490
:10329000FF0299C082E10E94811B892B09F493C02F
:1032A00080E090E00E94FF02109253038CC080E007
:1032B00090E00E94FF0205CF68E022CF851709F455
:1032C00022CF4F5F242F30E090E0F901EE5FFC4FFA
:1032D000DC01A752BD4F7C917083F901E053FD4F93
:1032E000708301968F710DCF2430B1F42091D002FC
:1032F00081ED92E0A3E0B3E0FC013E2F381B3217D2
:1033000018F431913D93F9CF87E3820F9091020336
:10331000892B8093020302CF80915303823069F49A
:103320009160909302035F9A5BEEE52E53E0F52ED9
:103330008E010F5F1F4FB80110C05F988091CD02C2
:10334000811103C081E08093CD028091CD02833052
:1033500059F784E08093CD02E7CFF70181917F0197
:1033600069A37AA30E94190DF801819391938F01AB
:1033700069A17AA1FBEFEF16F3E0FF0671F78091E8
:10338000C60343E053E087700E94FD03CACE882342
:1033900009F4CECE2091540331E0320F3093540320
:1033A0002913C6CE0CC010925603E2CE80913A0388
:1033B000883009F45F9A89E080933A03D9CE10925D
:1033C00054038150B5CEA296ECE00C9467251F9271
:1033D0000F920FB60F9211242F933F938F939F93C9
:1033E000AF93BF938091FE039091FF03A0910004DF
:1033F000B09101043091FD0323E0230F2D3720F419
:103400000196A11DB11D05C026E8230F0296A11D3E
:10341000B11D2093FD038093FE039093FF03A093BF
:103420000004B09301048091020490910304A091E0
:103430000404B09105040196A11DB11D80930204FE
:1034400090930304A0930404B0930504BF91AF913B
:103450009F918F913F912F910F900FBE0F901F90D2
:1034600018952FB7F8946091FE037091FF03809137
:103470000004909101042FBF08953FB7F894809104
:10348000020490910304A0910404B091050426B5B0
:10349000A89B05C02F3F19F00196A11DB11D3FBF8C
:1034A0006627782F892F9A2F620F711D811D911D1C
:1034B00042E0660F771F881F991F4A95D1F708953C
:1034C000CF92DF92EF92FF92CF93DF936B017C015B
:1034D0000E943D1AEB01C114D104E104F10479F01A
:1034E0000E943D1A6C1B7D0B683E7340A0F381E087
:1034F000C81AD108E108F108C851DC4FECCFDF91C0
:10350000CF91FF90EF90DF90CF900895789484B59D
:10351000826084BD84B5816084BD85B5826085BDCF
:1035200085B5816085BDEEE6F0E0808181608083B5
:10353000E1E8F0E010828081826080838081816098
:103540008083E0E8F0E0808181608083E1E9F0E061
:10355000808182608083808181608083E0E9F0E007
:10356000808181608083E1ECF0E0808184608083F1
:10357000808182608083808181608083E3ECF0E0E1
:10358000808181608083E0ECF0E0808182608083D4
:10359000E2ECF0E0808181608083EAE7F0E0808106
:1035A0008460808380818260808380818160808369
:1035B000808180688083089590E0FC013197EE302F
:1035C000F10590F5E35AFF4F0C947C258091800023
:1035D0008F7703C0809180008F7D80938000089555
:1035E00084B58F7702C084B58F7D84BD08958091A6
:1035F00090008F7707C0809190008F7D03C08091ED
:103600009000877F8093900008958091C0008F770D
:1036100003C08091C0008F7D8093C0000895809189
:10362000C200877F8093C2000895CF93DF9390E01C
:10363000FC01E75EFE4F2491FC01E95CFE4F8491A2
:10364000882349F190E0880F991FFC01EF58FE4F45
:10365000A591B4918D599E4FFC01C591D4919FB70E
:10366000611108C0F8948C91209582238C938881F5
:1036700082230AC0623051F4F8948C91322F309535
:1036800083238C938881822B888304C0F8948C9147
:10369000822B8C939FBFDF91CF910895A1E0B0E082
:1036A000E4E5FBE10C945325282F30E0F901E550C7
:1036B000FF4F8491F901E75EFE4F1491F901E95C37
:1036C000FE4F04910023C9F0882321F069830E94F2
:1036D000DC1A6981E02FF0E0EE0FFF1FED59FE4F7D
:1036E000A591B4919FB7F8948C91611103C0109586
:1036F000812301C0812B8C939FBF2196E4E00C9421
:103700006F25CF93DF93282F30E0F901E550FF4F6D
:103710008491F901E75EFE4FD491F901E95CFE4F17
:10372000C491CC2391F081110E94DC1AEC2FF0E0BF
:10373000EE0FFF1FEB5AFE4FA591B4912C912D2354
:1037400081E090E021F480E002C080E090E0DF9131
:10375000CF9108958091540490915504209156047E
:1037600030915704821B930B8F73992708952091F2
:1037700054043091550480915604909157042817B1
:10378000390749F0E0915604F0915704EC5EFB4F85
:10379000808190E008958FEF9FEF08952091540469
:1037A0003091550480915604909157042817390799
:1037B000A9F0E0915604F0915704EC5EFB4F808134
:1037C00020915604309157042F5F3F4F2F733327BA
:1037D000309357042093560490E008958FEF9FEFA5
:1037E0000895CF93DF93C0915404D091550421964E
:1037F000CF73DD278091560490915704C817D907DD
:1038000099F082E00E94A6208F3F2FEF920761F08F
:10381000E0915404F0915504EC5EFB4F8083D0930B
:103820005504C0935404DFCFDF91CF91089583E016
:103830000E94F1220895A1E0B0E0E1E2FCE10C94E5
:1038400053258C0169838091A401882359F041E0BC
:1038500050E0BE016F5F7F4F83E00E94D9201816B1
:1038600019063CF081E090E0F8019383828380E0C8
:1038700090E02196E4E00C946F25FC0120812E5FFE
:10388000208342E450E06FE771E080E80E94592114
:103890000895FC0181819081913A59F4813209F0B7
:1038A0004BC047E050E06DE971E080E00E94592193
:1038B00045C0913209F040C0803239F467E070E0D1
:1038C0008DE991E00E949D2139C0823209F034C017
:1038D00082818093A40180919D0190919E01A0918D
:1038E0009F01B091A001803B9440A105B10531F545
:1038F0008091A40180FD12C087E797E790930108AB
:10390000809300082BE088E190E00FB6F894A8952A
:10391000809360000FBE2093600010C088E10FB656
:10392000F89480936000109260000FBEA8951092EA
:1039300001081092000802C080E0089581E0089517
:103940000895109209041092080488EE93E0A0E014
:10395000B0E080930A0490930B04A0930C04B093FE
:103960000D048EE292E0909307048093060408957C
:10397000A0E0B0E0EEEBFCE10C944F256C017A0185
:10398000EB01E60EF71E00E010E0CE15DF0561F05A
:103990006991D601ED91FC910190F081E02DC60175
:1039A0000995080F191FF1CFC801CDB7DEB7E8E0C0
:1039B0000C946B256115710589F0DB010D900020D9
:1039C000E9F7AD0141505109461B570BDC01ED9160
:1039D000FC910280F381E02D0995089580E090E04C
:1039E0000895EF92FF920F931F93CF93DF938C0173
:1039F000FB01C0E0D0E064917F018FEFE81AF80A84
:103A0000662361F0D801ED91FC910190F081E02DE9
:103A1000C8010995C80FD91FF701EDCFCE01CDB769
:103A2000DEB7E6E00C946D250E94DA1C0895DC01F7
:103A3000ED91FC910190F081E02D099508950F938F
:103A40001F93CF93DF93EC016DE00E94171D8C0153
:103A50006AE0CE010E94171D800F911FDF91CF9168
:103A60001F910F9108950F931F93CF93DF93EC0154
:103A70000E94F11C8C01CE010E941F1D800F911F1E
:103A8000DF91CF911F910F9108950F931F93CF93C3
:103A9000DF93EC010E94DA1C8C01CE010E941F1DF5
:103AA000800F911FDF91CF911F910F9108950F9378
:103AB0001F93CF93DF93EC010E94171D8C01CE0161
:103AC0000E941F1D800F911FDF91CF911F910F91B9
:103AD0000895A1E2B0E0EFE6FDE10C944B257C01F6
:103AE000C42EE52FCB01D22E19A221E02D1510F006
:103AF0002AE0D22E8E010F5D1F4F8D2C912CA12C10
:103B0000B12C6C2D7E2FA50194010E9404258C2DD3
:103B1000D29E80191124015011098A3010F4805D61
:103B200001C0895CF80180832115310541055105EB
:103B300021F0C22EE32FCA01E4CFB801C7010E94D1
:103B4000DA1CA196ECE00C946725A0E0B0E0EBEA6B
:103B5000FDE10C944F25EC016A017B012115310533
:103B600041F4E881F9810190F081E02D642F0995FD
:103B70001DC02A303105A9F477FF12C06DE20E9402
:103B8000171D8C0144275527BA014C195D096E0990
:103B90007F092AE0CE010E94691D800F911F06C097
:103BA0002AE0B701A601CE010E94691DCDB7DEB79C
:103BB000E8E00C946B250F931F93CF93DF93EC01F8
:103BC0009A01AB01662757FD6095762F0E94A51DCF
:103BD0008C01CE010E941F1D800F911FDF91CF919C
:103BE0001F910F9108952115310549F4DC01ED91E4
:103BF000FC910190F081E02D642F099508950E94B9
:103C0000691D08959A01462F50E060E070E00E941F
:103C1000F31D08959A01AB0160E070E00E94F31D6E
:103C200008950F931F93CF93DF93EC019A01462FD2
:103C300050E060E070E00E94F31D8C01CE010E9414
:103C40001F1D800F911FDF91CF911F910F9108953C
:103C5000FC0124853585F901E05CFF4F808191816D
:103C6000F901EE5BFF4F20813181821B930B8F7333
:103C700099270895FC0184859585FC01E05CFF4F40
:103C800040815181FC01EE5BFF4F20813181421761
:103C9000530741F00190F081E02DE80FF91F80817A
:103CA00090E008958FEF9FEF0895FC01848595853E
:103CB000FC01E05CFF4F40815181FC01EE5BFF4F56
:103CC000208131814217530779F0A081B181A80F7B
:103CD000B91F8C91208131812F5F3F4F2F73332784
:103CE0003183208390E008958FEF9FEF0895FC01CA
:103CF00081A1882329F0A489B5898C9186FFFBCF07
:103D000011A20895CF93DF93FC0126853785D90151
:103D1000A05CBF4F8D919C91119701968F7399274D
:103D2000E901CE5BDF4F4881598184179507D9F3AC
:103D30000D90BC91A02DA20FB31F6C93A685B785E3
:103D4000A05CBF4F11969C938E93A689B7892C9146
:103D500081E090E0078C02C0880F991F0A94E2F777
:103D6000282B2C9381E081A30488F589E02D8081A4
:103D70008064808381E090E0DF91CF910895089581
:103D80001F920F920FB60F9211242F933F934F93D0
:103D90008F939F93EF93FF938091C80082FD1CC087
:103DA0004091CE008091FE049091FF0401968F73A4
:103DB000992720910005309101058217930771F032
:103DC000E091FE04F091FF04E254FB4F4083909396
:103DD000FF048093FE0402C08091CE00FF91EF911A
:103DE0009F918F914F913F912F910F900FBE0F9008
:103DF0001F90189588E594E00E94281E892B11F0E9
:103E00000E94BF1E08951F920F920FB60F921124A9
:103E10002F933F938F939F93EF93FF932091BA0437
:103E20003091BB048091BC049091BD0428173907E0
:103E300031F48091C9008F7D8093C90014C0E09156
:103E4000BC04F091BD04E658FB4F20818091BC0476
:103E50009091BD0401968F7399279093BD04809330
:103E6000BC042093CE00FF91EF919F918F913F91E1
:103E70002F910F900FBE0F901F901895A0E0B0E00B
:103E8000E4E4FFE10C944B25FC011382128288EEDE
:103E900093E0A0E0B0E084839583A683B78380E4B9
:103EA00092E0918380837587648757874687318B3B
:103EB000208B138B028BF58AE48AD78AC68AB18E4F
:103EC000A08E938E828E8F85848F8889858F898935
:103ED000868F8A89878F8B8980A3ECE00C94672575
:103EE000CF92DF92EF92FF92CF93DF93EC016A01C2
:103EF0007B01411581EE580761057105F9F0EC89E8
:103F0000FD8981E090E008A002C0880F991F0A9403
:103F1000E2F7808360E079E08DE390E0A70196010D
:103F20000E940425215031094109510956954795B0
:103F300037952795211580E1380798F0EC89FD89A0
:103F4000108260E874E88EE190E0A70196010E947B
:103F50000425215031094109510956954795379556
:103F60002795E889F9893083EA89FB89208319A29A
:103F7000EE89FF89408181E090E09C010C8C02C0B9
:103F8000220F331F0A94E2F7422B4083EE89FF8908
:103F900040819C010D8C02C0220F331F0A94E2F76E
:103FA000422B4083EE89FF8940819C010E8C02C028
:103FB000220F331F0A94E2F7422B4083EE89FF89D8
:103FC00020810F8C02C0880F991F0A94E2F7809518
:103FD00082238083DF91CF91FF90EF90DF90CF908D
:103FE00008958F929F92AF92BF92CF92DF92EF92FD
:103FF000FF920F931F9381E08F9385E08F9387E06B
:104000008F9383E08F9384E08F93EEEC8E2E912C30
:10401000FAECAF2EB12CA9ECCA2ED12CB8ECEB2EB9
:10402000F12C0CEC10E02DEC30E04AE754E06EEBA4
:1040300074E088E594E00E943E1F0F900F900F906F
:104040000F900F901F910F91FF90EF90DF90CF9006
:10405000BF90AF909F908F9008950E94861A82E043
:1040600095E00E94FB220E946214CAEFDEE10E94EA
:10407000F4162097E1F30E94FA1EF9CF615030F058
:104080002091F100FC0120830196F8CF289884E666
:104090008093090508952FB7FC012083F894677079
:1040A0006093E9000895A1E0B0E0E9E5F0E20C9446
:1040B0005525682FCE0101960E944B208091F20079
:1040C00099819FBF2196E2E00C947125A2E0B0E0B7
:1040D000ECE6F0E20C945225F62E8A019091080548
:1040E000992311F057FF03C08FEF9FEF2BC0682F6C
:1040F000CE0101967A830E944B208091F20090E0DD
:10410000A8017A81801791070CF4AC01EF2DF72FED
:10411000F40E84E6FE1639F02898809309059091F4
:10412000F1009193F7CF4115510521F08091F200F4
:10413000882321F089818FBFCA0104C08BE6809358
:10414000E800F8CF2296E5E00C946E25A1E0B0E0FF
:10415000ECEAF0E20C94552541E050E0BE016F5FBF
:104160007F4F0E946620019719F4898190E002C078
:104170008FEF9FEF2196E2E00C947125A1E0B0E073
:10418000E4ECF0E20C945525682FCE0101960E94D4
:104190004B209091E800892F807295FF04C0909188
:1041A000F20080E4891B99819FBF2196E2E00C9484
:1041B0007125A1E0B0E0EFEDF0E20C944725582E18
:1041C0007B01A42E952E80910805882369F0042F89
:1041D000152F8AEFB82E852D8072782E9AE3892EBE
:1041E000852D8074682E11C08FEF9FEF53C0852DF1
:1041F0000E94BE20482E81110CC0BA94A9F361E040
:1042000070E080E090E00E94601A0115110579F7D6
:1042100037C0282F30E0021713070CF4402EC42CAF
:10422000D12C0C191D09652DCE0101960E944B2041
:10423000772039F04A948FEF4816B1F01092F100D0
:10424000F9CFF701842D57FE07C0815058F09491A3
:104250009093F1003196F9CF815020F09191909395
:10426000F100FACFEC0CFD1C8091E80085FF0FC037
:104270000115110511F461100AC089818FBFC5CFE6
:104280005D9884E680930A058A2D992D03C080925B
:10429000E800F3CF2196E0E10C9463251092E90049
:1042A000109207051092060590930505809304056A
:1042B0000895CF93DF93FB0120E030E0DEEF241779
:1042C0003507A1F187FF02C0C49101C0C081A09150
:1042D0000605B09107056091040570910505A617C4
:1042E000B707B4F49091E8009570E1F39091E8007D
:1042F00092FD1EC0C093F100609106057091070504
:104300006F5F7F4F6F737727672B11F4D093E800AF
:1043100060910605709107056F5F7F4F70930705E9
:10432000609306052F5F3F4F3196C9CFC90102C088
:104330008FEF9FEFDF91CF910895A1E0B0E0E3EA26
:10434000F1E20C945425162F2091E80022FFFCCFB7
:10435000612F79830E943E208BEF8093E800812FAC
:104360007981972F2196E3E00C947025A1E0B0E0CD
:10437000ECEBF1E20C9455251982CE0101960E94D6
:104380003D1CCE0101960E949523898190E02196E3
:10439000E2E00C9471251F920F920FB60F92112438
:1043A000EF92FF920F931F932F933F934F935F933F
:1043B0006F937F938F939F93AF93BF93EF93FF93ED
:1043C000CF93DF93CDB7DEB76297DEBFCDBF10923C
:1043D000E9008091E80083FFE7C068E0CE010A961B
:1043E0000E943E2082EF8093E8009A8597FF05C0E7
:1043F0008091E80080FFFCCF03C08EEF8093E8003F
:10440000892F807609F0B5C08B85811105C0109287
:10441000F1001092F100C1C0282F2D7F213009F446
:10442000BCC0853049F48091E80080FFFCCF8C85CA
:1044300080688093E300B1C0863009F072C02D859A
:10444000E888F988223071F580E090E02A8B0E949C
:104450004E210E94B62199E08E010F5F1F4FF80197
:10446000392F11923A95E9F799832A892A8391E0A5
:104470009E8390E898879AEF99872091060530915E
:104480000705275F3F4F3C832B838D83C7010E9425
:104490004E2149E050E0B80180E00E9459210E947D
:1044A000B6217BC0C7012A8B0E944E212A89223265
:1044B00041F482E290E00E94A123892B09F06DC0B3
:1044C00070C0213069F488899989089711F4209384
:1044D000030580910305882389F066EC71E016C01E
:1044E000233009F05EC08C85882359F0823061F05A
:1044F000813009F056C06AEE71E008C068ED71E0E5
:1045000005C064E272E002C062E072E0611571050C
:1045100009F447C0FB01449150E080E80E94592112
:104520003CC0873009F43DC0883021F481E080939D
:10453000F10033C0893089F5937099F5E2ECF1E030
:1045400081E021E096E38093E9002093EB00349131
:104550003093EC009093ED008F5F3196853099F7A2
:104560008EE78093EA001092EA008C85809308051C
:1045700014C0888999890E944E218E85811105C0B9
:10458000CE010A960E94491C06C0823051F4CE0129
:104590000A960E94C323882321F08EEF8093E800BF
:1045A00003C081E28093EB0062960FB6F894DEBF01
:1045B0000FBECDBFDF91CF91FF91EF91BF91AF9132
:1045C0009F918F917F916F915F914F913F912F912B
:1045D0001F910F91FF90EF900F900FBE0F901F90C3
:1045E00018958093E9008091F200882319F08AE3FE
:1045F0008093E80008951092080581E08093D70029
:1046000080EA8093D80082E189BD09B400FEFDCF25
:1046100061E070E080E090E00E94601A80E98093A1
:10462000D8008CE08093E2001092E000559A209A26
:1046300008951F920F920FB60F9211242F933F935C
:104640004F935F936F937F938F939F93AF93BF939A
:10465000EF93FF938091E1001092E10083FF0FC080
:104660001092E90091E09093EB001092EC0092E33D
:104670009093ED001092080598E09093F00082FF6F
:1046800026C083E00E94F12282E00E94532088230A
:1046900021F086E094E00E94F11B80910A058823B6
:1046A00039F080910A05815080930A05882369F0CA
:1046B00080910905882359F08091090581508093E4
:1046C0000905811104C0289A02C05D9AF1CFFF91BB
:1046D000EF91BF91AF919F918F917F916F915F917A
:1046E0004F913F912F910F900FBE0F901F901895F3
:1046F000FF920F931F93CF93DF93EC01F62EE88187
:10470000F9810480F581E02D09958C01E881F9811A
:104710000680F781E02D6F2DCE010995C8019927FC
:10472000CDB7DEB7E5E00C946E25FC0120812F5F4C
:10473000208349E150E068EA72E080E80E94592154
:10474000089545E650E061EC72E080E80E9459214E
:104750000895A1E0B0E0EFEAF3E20C9451258983DB
:104760008B017A0141E050E0BE016F5F7F4F84E032
:104770000E94D920A701B80184E40E94D920219683
:10478000E6E00C946D25FC0191818081813A31F441
:1047900081E0913091F0933089F411C0813271F44D
:1047A0009B3021F482818093A60105C09A3031F4B8
:1047B00082818093A50181E00895089580E00895A5
:1047C000FC0110820895FC011382128220E532E080
:1047D00031832083089548E050E082E00E94A923BD
:1047E0000895CF93DF93DC01683818F0E8E7E60F0F
:1047F00025C0E62FF0E067FF11C0E058F10981E025
:1048000090E001C0880FEA95EAF714969C911497FE
:10481000982B14969C931497E0E010C0E85DFD4F30
:10482000E491EE2309F440C0E7FF08C014968C9190
:104830001497826014968C931497EF7716968C9148
:1048400016978E1741F117968C9117978E1719F1BD
:1048500018968C9118978E17F1F019968C911997DC
:104860008E17C9F01A968C911A978E17A1F01B9685
:104870008C911B978E1779F080E090E0ED01C80FC6
:10488000D91F2E81211102C0EE8305C0019686300A
:104890009105A1F709C0BD016C5F7F4FCD010E945A
:1048A000EB2381E090E008C081E090E013969C93B8
:1048B0008E93129780E090E0DF91CF910895683851
:1048C00018F0E8E7E60F25C0E62FF0E067FF12C01A
:1048D000E058F10921E030E001C0220FEA95EAF743
:1048E0002095DC0114963C911497322314963C9346
:1048F000E0E00FC0E85DFD4FE491EE2329F1E7FF12
:1049000008C0DC0114962C9114972D7F14962C93DB
:10491000EF7720E030E0EE2351F0DC01A20FB31F6F
:1049200016964C9116974E1302C016961C922F5F46
:104930003F4F2630310579F7BC016C5F7F4F0E94F5
:10494000EB2381E090E0089580E090E00895FC0181
:104950001682178210861186128613861482BC0175
:104960006C5F7F4F0E94EB23089587E195E00E94E2
:10497000E0238BE095E00E94E3230895A29FB0011D
:10498000B39FC001A39F700D811D1124911DB29F83
:10499000700D811D1124911D08950E94BE24A59FB4
:1049A000900DB49F900DA49F800D911D112408952A
:1049B000B7FF0C94CD240E94CD24821B930B089545
:1049C000DB018F939F930E94CD24BF91AF91A29F53
:1049D000800D911DA39F900DB29F900D11240895FD
:1049E00097FB072E16F4009407D077FD09D00E949C
:1049F000822507FC05D03EF4909581959F4F089540
:104A0000709561957F4F0895A1E21A2EAA1BBB1BDA
:104A1000FD010DC0AA1FBB1FEE1FFF1FA217B3078A
:104A2000E407F50720F0A21BB30BE40BF50B661FA0
:104A3000771F881F991F1A9469F760957095809564
:104A400090959B01AC01BD01CF010895052E97FB08
:104A50001EF400940E943D2557FD07D00E940425B6
:104A600007FC03D04EF40C943D25509540953095AD
:104A700021953F4F4F4F5F4F0895909580957095CA
:104A800061957F4F8F4F9F4F08952F923F924F9286
:104A90005F926F927F928F929F92AF92BF92CF92CE
:104AA000DF92EF92FF920F931F93CF93DF93CDB7D7
:104AB000DEB7CA1BDB0B0FB6F894DEBF0FBECDBF4F
:104AC00009942A88398848885F846E847D848C8420
:104AD0009B84AA84B984C884DF80EE80FD800C8129
:104AE0001B81AA81B981CE0FD11D0FB6F894DEBF0C
:104AF0000FBECDBFED010895EE0FFF1F0590F4919D
:104B0000E02D0994AA1BBB1B51E107C0AA1FBB1FC4
:104B1000A617B70710F0A61BB70B881F991F5A9549
:104B2000A9F780959095BC01CD0108958F929F9231
:104B3000AF92BF92CF92DF92EF92FF92CF93DF932B
:104B4000EC01688179818A819B81611571058105FC
:104B5000910521F464E279ED8BE597E02DE133EFE7
:104B600041E050E00E94262549015A019B01AC0119
:104B7000A7EAB1E40E94CD246B017C01ACEEB4EF56
:104B8000A50194010E94DB24C60ED71EE81EF91E63
:104B9000F7FE06C081E0C81AD108E10880E8F80AEB
:104BA000C882D982EA82FB82C701B6019F77DF9172
:104BB000CF91FF90EF90DF90CF90BF90AF909F90FC
:104BC0008F9008950E949625089586E091E00E94B6
:104BD000962508956093060170930701809308015C
:104BE000909309010895F999FECF92BD81BDF89A7D
:104BF000992780B50895262FF999FECF1FBA92BD47
:104C000081BD20BD0FB6F894FA9AF99A0FBE0196AD
:064C10000895F894FFCFA7
:104C160000001805200001000000FF00020002004D
:104C2600020002000200020002000200020002006E
:104C360002000200020002000200028025000005B8
:104C4600400AA1204EA50020244EA52C2330C012D8
:104C560000001A400AA1204EA5001B1E27522C2335
:104C6600308025000005400AA1204EA50020244ED4
:104C7600A52C2330004B000006400AD0009D4900B9
:104C86007B289D492C233000E1000005400A4501A0
:104C9600D7DC03B81E0EBF00232E48E801008A4069
:104CA6000A6001555502AD1E20000023C800E10030
:104CB6000000000000010154582074696D656F758D
:104CC600742100456E746572696E67206164617057
:104CD60074697665206368616E6E656C2073656CB9
:104CE600656374696F6E2C207069636B696E673AD1
:104CF600007363616E6E6572206D6F6465004F7040
:104D0600656E4C52536E67205458207374617274EA
:104D1600696E672000206F6E20485720006D6F6413
:104D2600756C65206C6F636B65643F0000070B0C48
:104D360010111500160A13223129000000001B1C51
:104D4600B81CAA1BCE1BB71B171CF11B00000000CA
:104D5600821EB81C281E551E3A1E771E0000000033
:0A4D66007823B81CF1235F24A72472
:1070000055C000006EC000006CC000006AC00000E7
:1070100068C0000066C0000064C0000062C00000DC
:1070200060C000005EC00000F2C400005AC0000052
:1070300058C0000056C0000054C0000052C00000FC
:1070400050C0000078C000004CC000004AC00000E2
:1070500048C0000046C0000044C0000042C000001C
:1070600040C000003EC000003CC000003AC000002C
:1070700038C0000036C0000034C0000032C000003C
:1070800030C000002EC000002CC000002AC000004C
:1070900028C0000026C0000024C0000022C000005C
:1070A00020C000001EC000001CC0000011241FBE34
:1070B000CFEFDAE0DEBFCDBF11E0A0E0B1E0E2E368
:1070C000FFE702C005900D92A83AB107D9F711E089
:1070D000A8EAB1E001C01D92AE3BB107E1F78FD342
:1070E00026C78ECFF89410926F00109281001092F4
:1070F00085001092840081E085BF15BE47985D9A97
:10710000289A0C94000008952091B2013091B301A7
:107110002F5F3F4F3093B3012093B201932F37FF7E
:1071200003C08EEF831B982F990F921710F4479886
:107130000895479A08951F920F920FB60F92112447
:107140002F938F939F93EF93FF931092850010924C
:1071500084008091A8019091A901009741F00197C6
:107160009093A9018093A801892B09F45D9A8091DD
:10717000AA019091AB01009741F001979093AB0168
:107180008093AA01892B09F4289AE0E0F0E0859128
:1071900094918F5F9F4F49F08091AC019091AD0128
:1071A00001969093AD018093AC01FF91EF919F9177
:1071B0008F912F910F900FBE0F901F90189584E024
:1071C0008093E9000DC08091E8008B778093E80000
:1071D00003C08EB3882351F08091E80082FFF9CF7D
:1071E0008091E80085FFEFCF8091F1000895982FFE
:1071F00083E08093E9008091E80085FD0DC08091D7
:10720000E8008E778093E80003C08EB3882369F08E
:107210008091E80080FFF9CF9093F1005D9884E6BB
:1072200090E09093A9018093A80108954F925F92F6
:107230006F927F928F929F92AF92BF92CF92DF9286
:10724000EF92FF920F931F93CF93DF9384E080938D
:10725000E9008091E80082FF57C2289884E690E018
:107260009093AB018093AA01AADF182F853481F493
:107270008CE49DE19093AD018093AC0107B600FCD6
:10728000FDCFF999FECF81E180935700E89503C0C7
:10729000843519F494DF8DE00DC28C34E1F3803530
:1072A000D1F3843721F484E4A2DF80E003C2813685
:1072B00011F489E5FFC18134B1F481DF182F7FDF3C
:1072C00090E0880F991FAA2797FDA095BA2F312F1C
:1072D000330F20E0442737FD4095542F822B932B0A
:1072E000A42BB52BB8C1803711F483E5E3C18335F6
:1072F00049F4C0E0D1E089917ADF21E0C730D207BC
:10730000D1F7D9C1863521F481E371DF80E3D2C1A1
:10731000833731F487E86BDF85E969DF8EE1CAC125
:107320008536B9F4E0E0F0E093E085E09093570013
:10733000E89507B600FCFDCF80935700E89507B6A7
:1073400000FCFDCFE058FF4FA0E7E030FA0771F7EF
:10735000A2CF823739F4E1E0F0E089E08093570072
:107360008491A8C1863439F4E0E0F0E089E08093AC
:10737000570084919FC18E3439F4E3E0F0E089E056
:1073800080935700849196C1813539F4E2E0F0E0B2
:1073900089E08093570084918DC1823631F489E56C
:1073A00026DF80E024DF80E885C1823419F087364B
:1073B00009F0E5C01092AD011092AC0100DF082F7A
:1073C000FEDEF82EFCDE682E8554823008F071C196
:1073D000902F80E0CF2DD0E0C82BD92B10926F00DA
:1073E000173609F04BC081E180935700E895DD2402
:1073F000CC24C3943FC0E090AE01F090AF01009167
:10740000B0011091B101B6E46B16D9F4ED2DF0E0A6
:10741000EE29FF29E4918E2FEADEDD2081F082E063
:1074200090E0A0E0B0E0E80EF91E0A1F1B1FE092FA
:10743000AE01F092AF010093B0011093B101DC24D2
:1074400018C0D801C701B695A7959795879559D5C6
:10745000CEDE82E090E0A0E0B0E0E80EF91E0A1F68
:107460001B1FE092AE01F092AF010093B0011093A8
:10747000B1012197209709F0BECF7DC08090AE0169
:107480009090AF01A090B001B090B10196E4691660
:1074900009F05DC083E0F40180935700E89507B6DA
:1074A00000FCFDCF54C0F6E46F1661F5772031F192
:1074B000E090AE01F090AF010091B0011091B101E8
:1074C0007EDED82ECC24852D90E08C299D29F701D5
:1074D0000C0140925700E895112482E090E0A0E072
:1074E000B0E0E80EF91E0A1F1B1FE092AE01F092F9
:1074F000AF010093B0011093B10102C060DE582EBD
:10750000742423C0E090AE01F090AF010091B0016F
:107510001091B10116950795F794E79450DE682F06
:10752000C701F7D48091AE019091AF01A091B00155
:10753000B091B1010296A11DB11D8093AE0190934F
:10754000AF01A093B001B093B101219704C05524BD
:10755000772444244394209709F0A5CF96E4691634
:1075600041F485E0F40180935700E89507B600FCEC
:10757000FDCF8DE03CDE82E080936F009CC08334C1
:1075800071F40091AE011091AF0119DE90E021E09D
:10759000F8010C0120935700E89511247CCE833626
:1075A00019F5E090AE01F090AF010091B00110919B
:1075B000B10105DEF701E16090E021E00C012093CC
:1075C0005700E895112482E090E0A0E0B0E0E80EDA
:1075D000F91E0A1F1B1FE092AE01F092AF0100934B
:1075E000B0011093B10157CE8D3661F4E091AE0138
:1075F000F091AF0185E080935700E89507B600FC55
:10760000FDCF49CE823551F4E091AE01F091AF014A
:1076100005911491812FEBDD802F4CC0843421F52E
:10762000E090AE01F090AF010091B0011091B10176
:1076300016950795F794E794C2DD682FC70169D4C2
:107640008091AE019091AF01A091B001B091B101D4
:107650000296A11DB11D8093AE019093AF01A0933E
:10766000B001B093B10117CE843609F5E090AE01B8
:10767000F090AF010091B0011091B101D801C701A4
:10768000B695A795979587953CD4B1DD82E090E0BB
:10769000A0E0B0E0E80EF91E0A1F1B1FE092AE0149
:1076A000F092AF010093B0011093B10104C08B318F
:1076B00011F08FE39CDD83E08093E9009091E80076
:1076C0008091E8008E778093E80095FF04C010C099
:1076D0008EB38823C9F08091E80080FFF9CF8091B4
:1076E000E8008E778093E80003C08EB3882361F0B2
:1076F0008091E80080FFF9CF84E08093E9008091D9
:10770000E8008B778093E800DF91CF911F910F9174
:10771000FF90EF90DF90CF90BF90AF909F908F90B1
:107720007F906F905F904F9008959091B601892F50
:107730008F77813249F58091B7018032A1F0813293
:1077400019F5913A09F58091E800877F8093E80068
:107750008DE091E067E070E00BD28091E8008B77DC
:107760008093E8000895913279F48091E800877F52
:107770008093E8008DE091E067E070E05DD2809159
:10778000E8008E778093E800089582E061EC42E0A3
:10779000B5D083E061E842E1B1D084E060E842E145
:1077A000ADC084B7877F84BF88E10FB6F89480931B
:1077B0006000109260000FBE20E880E090E00FB6FD
:1077C000F89420936100809361000FBE81E085BF33
:1077D00092E095BF3F9A209A559AE1E6F0E0208327
:1077E000108247985D9A289A109289008AEF8093B8
:1077F000880090936F0083E080938100F0C04091F7
:10780000000850910108109201081092000894B7E6
:1078100014BE88E10FB6F894809360001092600067
:107820000FBE292F30E0F901E270F07091FD18C011
:1078300090FF05C0859194918F5F9F4F81F423FF46
:107840000FC08091090190910A014817590741F032
:10785000E0E0F0E0859194918F5F9F4F09F042DC6A
:10786000A0DF78941092AD011092AC010CC0DEDC68
:1078700036D38091AC019091AD0181549F4110F0BD
:107880001092140141DC80911401882381F78091CA
:10789000E00081608093E00025DC80E090E00895C6
:1078A000FA01923049F0933061F09130F9F485E1BA
:1078B00091E022E130E01EC087E291E02EE330E06B
:1078C00019C0882329F485E691E024E030E012C055
:1078D000813029F489E691E022E230E00BC0823069
:1078E00029F48DE891E028E130E004C080E090E0E8
:1078F00020E030E091838083C90108958093E900FE
:107900008091EB0081608093EB001092ED0060931A
:10791000EC004093ED008091EE00881F8827881FBF
:1079200008958091B60188238CF403C08EB3882318
:10793000B1F08091E80082FFF9CF8091E8008B7769
:107940008093E80008958EB3882349F08091E80081
:1079500080FFF9CF8091E8008E778093E80008954A
:10796000EF92FF920F931F9345D04CD008ED10E09B
:10797000F80180818F778083808180688083808117
:107980008F7D808319BC1EBA1092B40180EEE82E60
:10799000F12CF70180818B7F8083F80180818160E9
:1079A000808380E060E042E0A9DFE1EEF0E08081EA
:1079B0008E7F8083E2EEF0E0808181608083808131
:1079C00088608083F70180818E7F8083F8018081C9
:1079D000806180831F910F91FF90EF900895E7EDF4
:1079E000F0E08081816080838AE482BF81E08093BF
:1079F000B501B6CFE8EDF0E080818E7F80831092F4
:107A0000E20008951092DA001092E10008951F92AA
:107A10000F920FB60F9211242F933F934F935F93C2
:107A20006F937F938F939F93AF93BF93EF93FF9346
:107A30008091DA0080FF1BC08091D80080FF17C0C2
:107A40008091DA008E7F8093DA008091D90080FFE8
:107A50000BC080E189BD82E189BD09B400FEFDCF84
:107A600081E08EBB3BD203C019BC1EBA37D28091D5
:107A7000E10080FF17C08091E20080FF13C0809179
:107A8000E2008E7F8093E2008091E200806180932B
:107A9000E2008091D80080628093D80019BC85E014
:107AA0008EBB1CD28091E10084FF2CC08091E2004B
:107AB00084FF28C080E189BD82E189BD09B400FE50
:107AC000FDCF8091D8008F7D8093D8008091E10018
:107AD0008F7E8093E1008091E2008F7E8093E200B0
:107AE0008091E20081608093E2008091B40188235C
:107AF00031F48091E30087FD02C081E001C084E0A1
:107B00008EBBECD18091E10083FF21C08091E20027
:107B100083FF1DC08091E100877F8093E10082E0B8
:107B20008EBB1092B4018091E1008E7F8093E100C2
:107B30008091E2008E7F8093E2008091E20080617C
:107B40008093E20080E060E042E0D8DEC7D1FF91A0
:107B5000EF91BF91AF919F918F917F916F915F91C5
:107B60004F913F912F910F900FBE0F901F9018953E
:107B70009C014091BC015091BD014617570718F474
:107B8000F90190E044C06115710511F0AB01F8CF27
:107B90008091E8008E778093E80040E050E0F0CFDD
:107BA0008EB3882309F444C0853009F443C0809122
:107BB000E80083FF02C081E008958091E80082FD23
:107BC00031C08091E80080FF22C08091F300909145
:107BD000F200782F60E0292F30E0262B372B07C0EA
:107BE00081918093F100415050402F5F3F4F4115EC
:107BF000510519F02830310598F390E0283031050F
:107C000009F491E08091E8008E778093E8004115B7
:107C1000510531F6992321F605C08EB3882341F032
:107C2000853041F08091E80082FFF7CF80E0089531
:107C300082E0089583E008959C016115710529F49F
:107C40008091E8008B778093E800F90126C08EB31D
:107C5000882391F1853091F18091E80083FF02C083
:107C600081E008958091E80082FFF1CF06C0809105
:107C7000F10081936150704059F02091F3008091A0
:107C8000F200322F20E090E0822B932B892B79F7A2
:107C90008091E8008B778093E80061157105B9F653
:107CA00005C08EB3882341F0853041F08091E80013
:107CB00080FFF7CF80E0089582E0089583E0089583
:107CC0000F931F93DF93CF9300D0CDB7DEB7E6EBD2
:107CD000F1E08091F100819381E0EE3BF807C9F774
:107CE00024DD8091E80083FFE4C08091B60190918B
:107CF000B701953009F46DC0963040F4913081F1B0
:107D0000913070F0933009F0D4C02AC0983009F453
:107D1000A3C0993009F4B2C0963009F0CAC07CC043
:107D2000803809F4C6C0823809F0C3C08091BA0116
:107D300087708093E9008091EB001092E900209118
:107D4000E800277F2093E80090E025E0969587954E
:107D50002A95E1F781708093F1001092F10087C0BD
:107D6000882319F0823009F0A4C08F71823009F0A5
:107D7000A0C08091B801882331F52091BA01277005
:107D800009F497C02093E9008091EB0080FF1BC0AD
:107D9000933021F48091EB00806213C08091EB005E
:107DA00080618093EB0081E090E002C0880F991F12
:107DB0002A95E2F78093EA001092EA008091EB00A6
:107DC00088608093EB001092E9008091E800877F43
:107DD00051C0882309F06DC01091B8011F770FB70B
:107DE000F8948091E800877F8093E8009ADD809185
:107DF000E80080FFFCCF8091E3008078812B8093A6
:107E0000E30080688093E300112311F482E001C055
:107E100083E08EBB0FBF4DC08058823008F049C050
:107E20008091B8019091B9016091BA01AE014F5FA4
:107E30005F4F36DDBC01009709F43BC08091E8003C
:107E4000877F8093E80089819A8192DE8091E800A3
:107E50008B778093E8002DC0803859F58091E80039
:107E6000877F8093E8008091B4018093F100809136
:107E7000E8008E778093E80054DD1BC08823C9F4A6
:107E80009091B8019230A8F48091E800877F8093A8
:107E9000E8009093B40145DD8091B401882331F46A
:107EA0008091E30087FD02C081E001C084E08EBBC9
:107EB0006CDC8091E80083FF0AC08091EB00806257
:107EC0008093EB008091E800877F8093E8000F901B
:107ED0000F90CF91DF911F910F91089508951F93F7
:107EE0008EB3882361F01091E9001092E90080912F
:107EF000E80083FF01C0E4DE17701093E9001F91D2
:107F00000895F999FECF92BD81BDF89A992780B561
:107F10000895262FF999FECF1FBA92BD81BD20BDCD
:107F20000FB6F894FA9AF99A0FBE01960895F8944C
:107F3000FFCF4341544552494E4100777700080036
:107F400000000000000801120110010200000841B9
:107F500023360001000201000109023E0002010077
:107F60008032090400000102020100052400100112
:107F7000042402040524060001070582030800FF0B
:107F800009040100020A00000007050402100001B4
:107F90000705830210000104030904220341007253
:107FA000006400750069006E006F0020004C0065E1
:107FB000006F006E006100720064006F0000001826
:107FC00003410072006400750069006E006F0020BC
:0A7FD000004C004C004300000000CC
:00000001FF
